:100000000C94E9010C9421020C9421020C9421021D
:100010000C9421020C9421020C9421020C942102D4
:100020000C9421020C9421020C9403200C94D520F2
:100030000C94E21A0C9421020C9421020C942102DB
:100040000C9421020C9421020C9421020C942102A4
:100050000C9421020C946A1B0C9421020C94210232
:100060000C9421020C9421020C9421020C94210284
:100070000C9421020C9421020C9421020C94210274
:100080000C9421020C9421020C9421020C94210264
:100090000C9421020C9421020C9421020C94210254
:1000A0000C9421020C9421020C942102EB04EB0429
:1000B000170517057F059D05B506B506A805410678
:1000C0005206520642216921612269216122B5212D
:1000D000D82161222F223E22290000003A003B0055
:1000E0003C003D003E003F00400041000000420057
:1000F0004300440045004B0035001E001F00200057
:1001000021002200230024002500260027002D00C6
:100110002E0035002A0049002B0014001A000800A8
:10012000150017001C0018000C00120013002F000F
:100130003000310000004C003900040016000700B8
:1001400009000A000B000D000E000F003300340000
:100150000000280000004E00E10064001D001B00AC
:1001600006001900050011001000360037003800A5
:10017000E500000052000000E000E300E2000000A3
:10018000000000002C00000000000000E600E40079
:100190005000000051004F0001000000010001006C
:1001A0000100010001000100010001000000010048
:1001B0000100010001000100010001000100010037
:1001C0000100010001000100010001000100010027
:1001D0000100010001000100010001000100010017
:1001E0000100010001000100010001000100010007
:1001F00001000100000001000100010001000100F8
:1002000001000100010001000100010001000100E6
:1002100000000100000001000100010001000100D8
:1002200001000100010001000100010001000100C6
:1002300001000000010000000100010001000000B9
:1002400000000000010000000000000001000100AB
:1002500001000000010001001E03420045004C00A7
:100260004C004100200053004F004C00440045006A
:10027000520045004400000010034B0042004400BF
:10028000460041004E005300000004030904090227
:100290003B00020100A0FA09040000010301010073
:1002A0000921110100012240000705810308000116
:1002B00009040100010300000009211101000122CD
:1002C000B6000705820320000112010002000000B1
:1002D00008424B070001000102000105010902A1CB
:1002E0000185020901A10005091901290815002548
:1002F0000195087501810205010930093115812533
:100300007F95027508810609381581257F9501754D
:10031000088106050C0A38021581257F95017508AC
:100320008106C0C005010980A101850319012AB712
:1003300000150126B700950175108100C0050C0954
:1003400001A101850419012AA002150126A0029528
:100350000175108100C005010906A1018506050788
:1003600019E029E7150025019508750181020507A7
:10037000190029EF1500250195F075018102050886
:1003800019012905950575019102950175039101E2
:10039000C005010906A101050719E029E715002597
:1003A00001950875018102950175088101050719FC
:1003B0000029FF150026FF00950675088100050835
:1003C00019012905950575019102950175039101A2
:1003D000C00011241FBECFEFDAE0DEBFCDBF04B6F0
:1003E00003FE18C08091D8029091D902A091DA0240
:1003F000B091DB028730904BA740B04B59F410927C
:10040000D8021092D9021092DA021092DB02E0E0D8
:10041000F8E3099511E0A0E0B1E0E0ECF6E402C0F9
:1004200005900D92A239B107D9F722E0A2E9B1E017
:1004300001C01D92A83DB207E1F70E94C3120C94BF
:100440005E230C9400006E9A0C947411CF93C82F05
:100450000E940203882329F0C1FD02C0769A01C0E0
:100460007698CF91089581E0089581E008950C94E5
:10047000350208950C9439021F93CF93DF9300D077
:1004800000D01F92CDB7DEB749835A836B8330917A
:10049000950189819A81311114C0662359F0222374
:1004A00049F00E94F208182F682F89819A810E94D2
:1004B0009B0803C00E94C608182F69817A81812F8A
:1004C00004C00E94F20869817A810F900F900F900A
:1004D0000F900F90DF91CF911F910C942E10FC0183
:1004E000262F408151816281738184810C943C026A
:1004F00081E00895CF93DF93EC0160E00E946F02EA
:10050000BE01DF91CF910C943A020C9423020C941B
:10051000721108950E9445070E9489022FEF84E31B
:100520009CE0215080409040E1F700C000000C9416
:10053000901B0F931F93CF93DF938C0161E00E9478
:100540006F02EC01B8010E943702882309F444C00D
:10055000B801CE010E9446168823F1F1B801CE0100
:100560000E942D198823C1F1B801CE010E944117C4
:10057000882391F1B801CE010E948918882361F186
:10058000F8018281882309F1CB358DE5D807C1F0C8
:1005900050F4C115FCE5DF0781F0CF3DDC45A9F43F
:1005A0000E94290E19C0CC35EDE5DE0761F0CD358E
:1005B000DD4559F40E946C0D08C00E948A020CC0EF
:1005C0000E94750D02C00E94780DC801DF91CF9185
:1005D0001F910F910C94330280E0DF91CF911F9116
:1005E0000F9108950E94C41A80E00E947B160C941B
:1005F0000E030E946A150E9411030C94CA1A0895F2
:100600000C94FF0281E008950895CF93C82F0E94B3
:1006100000038C2F0E942602CF91089580E00C9455
:1006200005030E9489190C9405030E948919909171
:100630009401891721F0809394010C940503089587
:10064000CF93DF93CDB7DEB72B970FB6F894DEBF0D
:100650000FBECDBF4F83588769877A878B8761111B
:100660000E94B80C9E012F5F3F4F86E0F901119266
:100670008A95E9F785E0FE013796D90101900D9240
:100680008A95E1F789819A814C815D81452B31F012
:100690009F3F31F491E08F3F19F403C091E001C016
:1006A00090E090FF09C049815A816B817C818D81E6
:1006B0009E810E94D90B05C0C9010E947802811158
:1006C000F2CF2B960FB6F894DEBF0FBECDBFDF91F1
:1006D000CF910895FC01808191810E943409089591
:1006E000CF93882309F4A4C0C82F8238C1F40E9494
:1006F000891981FD9DC069E38091020190910301F8
:100700000E947F1A0E94DA0C2FEF81EE94E02150B4
:1007100080409040E1F700C0000069E319C08338D1
:1007200001F50E94891980FD83C063E58091020173
:10073000909103010E947F1A0E94DA0C2FEF81EE44
:1007400094E0215080409040E1F700C0000063E554
:1007500080910201909103010E948A1ACF910C941A
:10076000DA0C8438C1F40E94891982FD61C067E403
:1007700080910201909103010E947F1A0E94DA0C7D
:100780002FEF81EE94E0215080409040E1F700C0CF
:10079000000067E4DDCF8CEF8C0F813AD0F46C2F32
:1007A00080910201909103010E94FF19882349F072
:1007B0006C2F80910201909103010E948A1A0E947D
:1007C000DA0C6C2F80910201909103010E947F1A34
:1007D000C5CF80E28C0F883048F4C77081E001C03B
:1007E000880FCA95EAF70E949B0CB8CFEBE5EC0F97
:1007F000E33040F4F0E0E95BFE4F808190E0CF9180
:100800000C94BD19E8E5EC0FE73150F4F0E0EE0F81
:10081000FF1FE75EFE4F80819181CF910C94D31929
:10082000CD3E30F08C2F0E944813CF910C941A14B7
:10083000CF910895882309F464C0823879F40E9426
:10084000891981FF5EC069E38091020190910301E3
:100850000E947F1A0E94DA0C69E310C08338B1F459
:100860000E94891980FF4DC063E58091020190913B
:1008700003010E947F1A0E94DA0C63E58091020155
:10088000909103010E948A1A0C94DA0C843879F44E
:100890000E94891982FF35C067E48091020190911E
:1008A00003010E947F1A0E94DA0C67E4E7CF9CEFF5
:1008B000980F913A10F4682FE1CF90E2980F98309A
:1008C00050F4877091E001C0990F8A95EAF7892F5B
:1008D0000E94A10CD9CF9BE5980F933020F480E0C3
:1008E00090E00C94BD1998E5980F973120F480E0C2
:1008F00090E00C94D3198D3E20F00E94A3130C9429
:100900001A1408951F93CF93DF93182FEB010E94C1
:100910007003209741F08FE99FE00197F1F700C045
:1009200000002197F6CF812FDF91CF911F910C947A
:100930001A04893319F060E070E002C060E570E0ED
:100940000C948204882321F00E949B0C0C94DA0CF6
:100950000895882321F00E94A10C0C94DA0C0895CC
:10096000CF92DF92EF92FF920F931F93CF93DF937B
:100970007C01D62FC72FFC011281058102950F70D3
:100980000E94910C8823B9F01123A9F08C2F807F4D
:10099000803421F080E28D0F883068F08091AD02C4
:1009A00082FD09C082E00E943A0D0E94910C91E004
:1009B000D82ED92601C0D12CCC2EC2948FE0C822CB
:1009C0008C2D90E08C30910508F0CFC1FC01EA5AE3
:1009D000FF4F0C94EF228C2F807FCF70882311F073
:1009E000C295C07F112399F0CC2309F4AAC180E2FB
:1009F0008D0F883010F0D11104C08C2F0E949B0CF9
:100A000003C08C2F0E94AB0C0E94DA0C9AC18D2F70
:100A10000E941A04CC2309F4A8C180E28D0F88300B
:100A200038F1DD2329F18C2F0E94B10C24C08C2FCA
:100A3000807FCF70803211F0C295C07FDD2319F026
:100A4000D130A1F13DC08091AD0282FF17C01123CA
:100A500049F0CC2329F08C2F0E949B0C0E94DA0CC9
:100A600080E070C180E00E941A04CC2309F47DC1AB
:100A70008C2F0E94A10C0E94DA0C77C1112371F017
:100A8000002341F0013031F40E94BB0C8C2B0E94FA
:100A9000C30C6BC10E94BB0C8C2B1DC0002319F032
:100AA000013009F462C10E94D00C25C0112321F04D
:100AB000063008F05AC10EC0053008F056C11BC000
:100AC000112361F0002331F0F701858180FF39C1E6
:100AD0008F7085838C2F0E94A20447C1002359F098
:100AE000D93309F03FC1FFEF07EE13E0F1500040AA
:100AF0001040E1F735C18C2F0E94A90436C18C2F1C
:100B000086958695837019F0813061F02EC111238E
:100B100021F08D2F9C2F937002C080E090E00E9406
:100B2000BD192BC1112321F08D2F9C2F937002C072
:100B300080E090E00E94D31920C18D2F112319F07D
:100B40000E94481302C00E94A3130E941A1415C1E8
:100B50008C2F837009F047C011110BC12D2F2295E6
:100B600026952770220F220F6D2F6F70862F90E031
:100B7000A0E0B0E0022E04C0880F991FAA1FBB1F7F
:100B80000A94D2F7D4FF10C04FE050E060E070E06C
:100B900004C0440F551F661F771F2A95D2F7409552
:100BA00050956095709503C040E050E0BA01C6953D
:100BB000C695C3708A019B01082B192B2A2B3B2B4E
:100BC000C901B801C23049F058F4C13019F00E948F
:100BD000B107CFC00E949F07CCC00E94C307C9C005
:100BE0000E949D07C6C0112319F08C2F817001C08F
:100BF0008695882309F4BDC02D2F22952695277050
:100C0000220F220F6D2F6F70862F90E0A0E0B0E0D2
:100C1000022E04C0880F991FAA1FBB1F0A94D2F787
:100C2000D4FF10C04FE050E060E070E004C0440F1B
:100C3000551F661F771F2A95D2F7409550956095EE
:100C4000709503C040E050E0BA01C695C695C370E8
:100C50008A019B01082B192B2A2B3B2BC901B801B8
:100C6000C23049F058F4C13019F00E94760881C0B2
:100C70000E9464087EC00E9488087BC00E94D7073B
:100C800078C0CF70112339F08C2F0E94FD078D2F73
:100C90000E94A2046EC08D2F0E94A9048C2F0E9476
:100CA0001E0867C0D23F21F128F4D03F41F0D13F68
:100CB000C1F043C0D33F19F1D43F79F03EC01123B6
:100CC00041F0053008F051C08C2F8F710E9443080D
:100CD0004CC0063008F049C0F7CF8091AD0282FFCA
:100CE00018C0112339F08C2F8F710E94FD073DC071
:100CF0001123C9F38C2F8F710E941E0836C0112357
:100D000029F08C2F8F710E94E8072FC00E94E30703
:100D10002CC0112349F0CF718C2F0E94FD0763E096
:100D20008C2F0E941F0D21C081E00E943A0D0230DD
:100D3000E0F082E00E943A0D18C0112331F0002348
:100D400091F28D2F0E94700310C0002399F2D933C5
:100D500049F41FEF27EE33E0115020403040E1F717
:100D600000C000008D2F0E941A0488EF8C0D843083
:100D700020F40E9489190E940503DD20C9F00E9419
:100D80008D0C80FD15C0F70112820E94870C0E9415
:100D9000FD07C7010E94F9060E94870CDF91CF91E1
:100DA0001F910F91FF90EF90DF90CF900C941E0851
:100DB000DF91CF911F910F91FF90EF90DF90CF9037
:100DC00008950F931F93CF93DF93EC01688179818E
:100DD0008A810E943F098C010E949A080E948B0719
:100DE000B801CE010E94B004DF91CF911F910F9105
:100DF0000895CF93DF93EC01988189812B813C8109
:100E0000232B31F08F3F31F481E09F3F19F403C071
:100E100081E001C080E080FD1DC0CE010E949902EA
:100E2000811110C00E94910C8823A1F08A8188232F
:100E300089F08091AD0282FD0DC082E0DF91CF91FB
:100E40000C943A0DCE010E94E106CE01DF91CF91C4
:100E50000C947A02DF91CF91089580E090E00E9497
:100E6000BD1980E090E00E94D3190E94B80C0E9446
:100E7000DA0C0E944B150C941A1480910201909187
:100E800003010E94951A0C942D070E94A80C0C9443
:100E90003D0792959F70963079F010F4925001C002
:100EA0009A50923068F4803F69F018F4883E40F41C
:100EB00009C0843F29F406C0883E20F0813F11F02C
:100EC00080E0089581E00895FC01808191810E9475
:100ED00034090E9449070895CF93DF9300D000D0D2
:100EE0001F92CDB7DEB70F900F900F900F900F901D
:100EF000DF91CF910895CF93DF9300D000D000D041
:100F0000CDB7DEB726960FB6F894DEBF0FBECDBFC5
:100F1000DF91CF910895089508950C948C070C9457
:100F20008D070E948F076093D6017093D70180933D
:100F3000D8019093D9010C942D070C9491070F932D
:100F40001F930091D6011091D7012091D8013091C3
:100F5000D901602B712B822B932B1F910F910C9435
:100F600091070F931F930091D6011091D701209103
:100F7000D8013091D90160237123822393231F91DB
:100F80000F910C9491070F931F930091D60110912C
:100F9000D7012091D8013091D9016027712782278C
:100FA00093271F910F910C9491070C948C070E942A
:100FB000D5076093D2017093D3018093D4019093AD
:100FC000D5010C942D0760E070E0CB010C94D7079D
:100FD0000F931F9341E050E060E070E08A019B01B5
:100FE00004C0000F111F221F331F8A95D2F7C901B9
:100FF000B8011F910F910C94D7070F931F9341E0F5
:1010000050E060E070E004C0440F551F661F771F7A
:101010008A95D2F78091D2019091D301A091D40109
:10102000B091D5018A019B01082B192B2A2B3B2B50
:10103000C901B8011F910F910C94D7070F931F930B
:1010400041E050E060E070E004C0440F551F661FAF
:10105000771F8A95D2F7409550956095709580914D
:10106000D2019091D301A091D401B091D5018A0110
:101070009B01082319232A233B23C901B8011F918F
:101080000F910C94D7070F931F9341E050E060E05D
:1010900070E004C0440F551F661F771F8A95D2F772
:1010A0008091D2019091D301A091D401B091D5014A
:1010B0008A019B01082719272A273B27C901B80164
:1010C0001F910F910C94D7070F931F930091D2019A
:1010D0001091D3012091D4013091D501602B712B57
:1010E000822B932B1F910F910C94D7070F931F9373
:1010F0000091D2011091D3012091D4013091D501FA
:1011000060237123822393231F910F910C94D7079F
:101110000F931F930091D2011091D3012091D4011C
:101120003091D50160277127822793271F910F9156
:101130000C94D707089520E1929F800D1124E82F89
:10114000E695E695E695877051E001C0550F8A95C2
:10115000EAF785E0E89FF0011124EA56FE4F20E00F
:1011600030E070E04081CB01022E02C09695879559
:101170000A94E2F7817081958427852384278193DF
:101180002F5F3F4F2530310569F7089520E1929F89
:10119000800D1124682F669566956695982F977037
:1011A00085E0689FB001112440E050E080E0FB0141
:1011B000E40FF51FEA56FE4F208130E0092E02C0F1
:1011C000369527950A94E2F721703327042E01C043
:1011D000220F0A94EAF7822B4F5F5F4F453051058B
:1011E00031F70895BF92CF92DF92EF92FF920F9363
:1011F0001F93CF93DF938C01C090D201D090D30185
:10120000E090D401F090D5018091D6019091D70162
:10121000A091D801B091D901C82AD92AEA2AFB2A7B
:10122000CFE1D0E0D701C6010C2E04C0B695A7953A
:10123000979587950A94D2F780FD04C0219790F77F
:10124000B12C07C0BC2EB8018C2F0E94431001970F
:10125000A9F38B2DDF91CF911F910F91FF90EF900C
:10126000DF90CF90BF900895CF93DF93EC010E9461
:10127000F208BE010E944310DF91CF9108951F93A1
:10128000CF93DF93EB0190919501992321F0CB014E
:101290000E94340913C0882349F0CB010E94F20850
:1012A000182F682FCE010E949B0804C0CB010E941A
:1012B000C608182FBE01812F0E944310DF91CF91E5
:1012C0001F9108951F93CF93DF93C091DA0116E029
:1012D0008091DB01C81799F0D0E01C9FF0011D9FA1
:1012E000F00D1124E452FE4F4081518162817381DF
:1012F000848195810E947B072196C770E9CFDF9199
:10130000CF911F91089540910C0250910D02609170
:101310000E0270910F0280911002909111020C94B4
:101320007B07EF92FF920F931F93CF93DF938091F0
:10133000110282958F7009F065C080910E0288239A
:1013400009F460C08091DA01F090DB0110910C0289
:1013500000910D0260910F027091100291E01F3F09
:1013600009F090E0C0910001D0910101292F96E091
:10137000E92E8F1509F446C06115710521F00F3F64
:1013800021F030E003C031E001C0322F90E030FDA9
:1013900036C0E89EF001E99EF00D1124DF01A45251
:1013A000BE4F11963C911197301329C03C913113D7
:1013B00026C012963C911297311121C013964D917F
:1013C0005C911497461B570B4C175D07C0F4809136
:1013D00011028F70806180931102EF51FE4F808166
:1013E0008F70806180838CE092E00E94F906DF912B
:1013F000CF911F910F91FF90EF900C94620901968D
:101400008770B7CFDF91CF911F910F91FF90EF9031
:1014100008959F92AF92BF92CF92DF92EF92FF9288
:101420000F931F93CF93DF93CDB7DEB761970FB6BE
:10143000F894DEBF0FBECDBF8C0185E0F801DE0160
:101440001D9601900D928A95E1F7D8011296EC90C5
:1014500090910C02E0910D0220910F023091100248
:101460002115310531F0EF3F31F481E09F3F19F450
:1014700003C081E001C080E0B82FB1709B2E80FDD9
:1014800047C1D8014C9111965C9111971396AD907C
:10149000BC9014978CE0C82E82E0D82EF0900E02FB
:1014A000B501621B730B2091000130910101FF20F7
:1014B00009F4D9C0809111026217730708F095C032
:1014C000282F207F09F052C05E1313C0491311C0AA
:1014D000FE2CE1100EC08F708061809311020E947B
:1014E0008309C6010E94F90680911102F8018583E3
:1014F0004DC1AB2831F05F3F31F481E04F3F19F42B
:1015000003C081E001C080E080FD03C081E08E2542
:1015100002C080E090E0F82FF170FF2E80FF1CC029
:101520008091DA012091DB0136E0821709F40BC1CA
:1015300090E0389FF001399FF00D1124E452FE4FE6
:101540006181561306C06081461303C06281E612B2
:1015500003C001968770E9CFFE2CEE2009F416C176
:101560008091110281608093110254C05E1306C005
:10157000491304C0E11002C0F80199C0C8010E94DB
:101580006407882361F1EE2051F120911102822F2E
:1015900082958F7090E0029774F080910C02909188
:1015A0000D0298878F831986BB86AA862C87CE0169
:1015B00007960E94F90686E0F801ACE0B2E00190DF
:1015C0000D928A95E1F70E9491090E9483090AC051
:1015D0005E1711F1C8010E94640781112CC0C80177
:1015E0000E94F906FF24F394D1C0282F207F81F7B1
:1015F0007A2DB98AA88A6E2D89890E946C078CE0A1
:1016000092E00E94F90686E0D6011D928A95E9F7DC
:101610000E948309F12CBAC04913DCCFE110DACF64
:10162000F8018583C8010E94F90686E0D6011D9263
:101630008A95E9F7ABC0EE2091F220911102822F3A
:1016400082958F7090E002970CF4B5CF80910C02D8
:1016500090910D029A8389831B82BD82AC822E8376
:10166000CE010196A6CF6217730708F044C0FE2C86
:10167000EE2009F4B4CF5E1330C049132EC0209180
:10168000110220FD21C0822F82958F70482F50E0DB
:1016900041155105C9F0F80125834F30510541F03E
:1016A0008F5F982F9295907F822F8F70892B8583E3
:1016B000C8010E94F90686E0F801ACE0B2E00190B2
:1016C0000D928A95E1F73CC086E0F801ACE0B2E00B
:1016D00001900D928A95E1F759C0C8010E946407F4
:1016E000811169CF80911102816080931102C8013C
:1016F0000E94F9064BC07A2DB98AA88A6E2D898975
:101700000E946C0786E0D6011D928A95E9F718C001
:10171000EE2009F464CFC8010E946407F82E8823E4
:1017200009F45DCF86E0F801ACE0B2E001900D92E3
:101730008A95E1F78CE092E00E946A030E94910989
:101740000E94830923C04D875E878D859E850E94F8
:101750003409292F22952F70223028F49F7039F0F8
:10176000811105C00BC0243028F49F7049F4805EBD
:10177000883020F0C8010E94F9069F2CF92C06C081
:10178000D80115969C91907F91F7F8CF8F2D619697
:101790000FB6F894DEBF0FBECDBFDF91CF911F9182
:1017A0000F91FF90EF90DF90CF90BF90AF909F9000
:1017B00008951F93CF93DF93CDB7DEB72C970FB665
:1017C000F894DEBF0FBECDBF4F83588769877A87F5
:1017D0008B879C87CE0107960E94090A8823D1F047
:1017E0009F8188852A853B85232B31F08F3F31F4FB
:1017F00081E09F3F19F403C081E001C080E080FDDB
:1018000047C04F81588569857A858B859C850E9464
:101810007B073EC086E0FE013796DE0111960190FF
:101820000D928A95E1F7FF81E8856A857B856115D0
:10183000710531F0EF3F31F481E0FF3F19F403C04F
:1018400081E001C080E080FD23C02091DB0130E019
:10185000C9010196877099274091DA0150E08417F9
:101860009507F1F1F983EA837D836C8396E0929F7B
:10187000D001939FB00D1124A452BE4FFE013196AA
:1018800001900D929A95E1F78093DB010E94620925
:1018900016E08091DA019091DB01891771F1189FB0
:1018A000C001112484529E4F0E94090A882329F105
:1018B000E091DA011E9FF0011124E452FE4F4081B5
:1018C000518162817381848195810E947B0780911F
:1018D000DA0190E00196877099278093DA01D9CFD9
:1018E0000E9445071092DB011092DA01ECE0F2E071
:1018F00086E0DF011D928A95E9F72C960FB6F894E1
:10190000DEBF0FBECDBFDF91CF911F9108958091B3
:10191000320285958595859508958091320287706C
:10192000089590913202977081E009F480E0089563
:1019300080915502089590915502892B809355020C
:1019400008958095909155028923809355020895BA
:1019500010925502089590915402892B809354025D
:10196000089580959091540289238093540208959C
:1019700010925402089580913302089508950C94B2
:10198000BE0C0C94BF0C9091AD0292FD08C09091DA
:101990003302981721F0809333020C94C10C089500
:1019A00080913302882329F01092330280E00C9456
:1019B000C10C0895CF93DF93E0910201F0910301F0
:1019C000809155028083E0910201F09103019081A2
:1019D00080915402892B808380913302882381F087
:1019E000E0910201F09103019081892B8083809125
:1019F0000201909103010E94E91981110E94D00C0B
:101A0000C0910201D091030140E250E062E172E036
:101A1000CE010E940F23892B69F080E2FE01A2E132
:101A2000B2E001900D928A95E1F7CE01DF91CF915E
:101A30000C949519DF91CF9108950C94BE0C909160
:101A4000AD0292FD10C098E0899F90011124262BD1
:101A5000209332020E94FD07809132028595859580
:101A600085950C941D0D0C94FD071092320280E0B8
:101A70000C941D0D209132028095822380933202B6
:101A8000982F977099F430E0482F082E000C550BD2
:101A90002417350759F09091AD0292FD07C0859546
:101AA000859585950E941E080C94350D089590919A
:101AB000AD0292FB222720F9281769F080FB92F9EA
:101AC0009093AD028091AC029091AD020E94A50D61
:101AD00082E00C943A0D08958091AD0282FB882734
:101AE00080F991E089270C94570D81E00C94570DF3
:101AF00080E00C94570D6FEF7FEF80E090E00C9446
:101B0000482380E090E00E94242321E0893E9E4FFC
:101B100009F020E0822F089582E090E00C941C23CD
:101B200083E090E00C941C23CF9384E090E00E942B
:101B30001C23C82F82E290E00E941C232C2F30E04F
:101B4000A901582BCA01CF910895CF93C92F682FAF
:101B500084E090E00E942A236C2F82E290E0CF91F3
:101B60000C942A23AB01BC018FE090E00C943C2341
:101B7000AB01BC0183E190E00C943C2360E070E099
:101B8000CB010C94B80D60E070E0CB010E94B20D67
:101B90000C94BE0D69EE7EEF80E090E00E94482339
:101BA00060E082E090E00E942A2360E083E090E021
:101BB0000E942A231092D6011092D7011092D801C8
:101BC0001092D90160E084E090E00E942A2360E056
:101BD00082E290E00E942A2360E085E090E00E948B
:101BE0002A2360E086E090E00E942A236FEF87E0DE
:101BF00090E00E942A2340E050E0BA0188E090E0A3
:101C00000E943C2360E08DE090E00E942A2340E0A7
:101C100050E0BA0188E190E00E943C2360E087E157
:101C200090E00E942A2340E050E0BA018CE190E06D
:101C30000E943C2360E070E080E290E00E94482334
:101C400040E050E0BA0188E190E00E943C230C940F
:101C5000C30D0C94CA0D682F8EE090E00C942A23DB
:101C60000E944F1B60936602709367028093680224
:101C7000909369026093620270936302809364029E
:101C800090936502089585B7806885BF85B78068A1
:101C900085BF089581E008950C944A0E08950C9430
:101CA0004E0E0C944E0E0C94510E0C944E0E0C9441
:101CB000550E0C944E0E0E94430E8FE191E10E944E
:101CC0007F190E94590E0C94570E0E944F0E0C94CF
:101CD0004E0E0E9439110E9404030C9431170E9489
:101CE0003A1B0E941C120E94690E0E946A150C94F5
:101CF000530E5F926F927F928F929F92AF92BF929C
:101D0000CF92DF92EF92FF920F931F93CF93DF93C7
:101D1000CDB7DEB72A970FB6F894DEBF0FBECDBFA2
:101D20000E943112C82E81110E94300E36E5832E9A
:101D300032E0932E00E010E0502E802F0E945D11C3
:101D40005C01F401619071904F016826792661145D
:101D50007104B1F40F5F1F4F0630110569F78FEF63
:101D600089838A831B820E94431B8160782F9D8315
:101D70008C8349815A816B818D810E9420033AC0F6
:101D800080916A0281FD0E946611D12CEE24E394B9
:101D9000F12CC3018E219F21892B29F10E944C0E29
:101DA0008823A9F0DE825F82AE20BF2081E0AB28CD
:101DB00009F480E088870E94431B8160782F9A870E
:101DC00089874E815F8168858A850E942003000F84
:101DD000111FF801EA5AFD4F80819181E826F9260A
:101DE000F182E08207C0D394EE0CFF1CF0E1DF1219
:101DF000D0CFB0CF81E0C11001C080E02A960FB6ED
:101E0000F894DEBF0FBECDBFDF91CF911F910F9130
:101E1000FF90EF90DF90CF90BF90AF909F908F900A
:101E20007F906F905F9008950E94790E0E94301706
:101E30000E9438140C941503CF93DF930E9448102E
:101E4000EC01811521E5920708F045C0811530E5C8
:101E5000930708F094C0883E910528F5803E9105CF
:101E600008F0F8C0883A910570F4853A910508F0B9
:101E70007CC08130910509F475C008F4E8C004976E
:101E800008F0E8C0E4C08F3B910508F0E0C0C85AF4
:101E9000D0E0CC0FDD1FC65BDE4F0990D881C02D8E
:101EA000CE019464D8C0811540E2940758F481159E
:101EB00051E0950708F0CEC08D3E910508F4C7C0EB
:101EC0009065C9C0C11580E4D80708F4C0C0DF70B0
:101ED000CE01906AC0C0811525E59207A8F481154E
:101EE00034E5930708F095C0811543E5940708F0A1
:101EF0007BC0811552E5950708F061C0D82FCC272B
:101F0000CE01816F906AA7C0C11589E5D807A0F4FA
:101F1000C11528E5D20708F082C0C11536E5D30700
:101F200008F095C08C2F0E94DC108F7190E0D82FA4
:101F3000CC27CE0190628FC0C1154AE5D40708F4C2
:101F400074C0CE0190568115904208F080C08D2F4C
:101F50008F710E94DC10DD27D0628F71AE01582B8B
:101F6000CA0179C081E090E076C0C55AD0E0C85877
:101F7000DE4F8881C82FD0E0CE0190646CC074E041
:101F8000969587957A95E1F7282F23703C2F33702B
:101F900081E090E002C0880F991F3A95E2F79C68B3
:101FA000AC01522B9A019C2F9F709695969550E20A
:101FB000959FE0011124C9018C2B9D2B4CC083708F
:101FC000992721E030E002C0220F331F8A95E2F703
:101FD0009C2F9695969580E2989FE0011124C22B44
:101FE000D32BCE019C6837C08370992721E030E065
:101FF00002C0220F331F8A95E2F79C2F9695969583
:1020000040E2949FE0011124C22BD32BCE019A68A9
:1020100022C0D82FCC27CE01846F906A1CC0DC2F41
:10202000CC27CE01806F906A16C08C2F8F700E94D3
:10203000DC1094E0D695C7959A95E1F7CF70D0E083
:10204000DC2FCC27D0699E01282BC90104C080E079
:1020500090E001C0CE01DF91CF910895E72FF0E02D
:1020600096E0899FE00DF11D112484E0EE0FFF1F23
:102070008A95E1F7E60FF11DEE0FFF1FE852FF4FC3
:102080008591949108950E942E100E941C0F08952E
:102090008238910569F1B0F48133910509F46DC07E
:1020A00048F48932910509F463C08A32910509F434
:1020B00069C008958533910509F455C089339105A8
:1020C000B9F00895833E910569F138F4803E910599
:1020D000B1F0823E910509F10895863E9105A9F17E
:1020E000873E9105B9F1843E910509F064C023C093
:1020F0002091AC0220FD4FC021FD4DC0089580917C
:10210000AC0280FD44C08091AD0280FF44C080914C
:10211000AC0284FD42C083EE4DC08091AC0282FFD0
:1021200038C0F5CF8091AC0282FD33C08091AD0202
:1021300080FD31C0ECCF8091AD0281FF32C0809133
:10214000AC0284FD2AC087EE35C08091AC0283FFCB
:1021500026C0F5CF8091AC0283FD21C08091AD02F5
:1021600081FD1FC0ECCF8091AC0285FD1CC01DC05D
:102170008091AC0285FD19C016C08091AC0286FD2D
:1021800016C017C08091AC0286FD13C010C089E351
:1021900011C082EE0FC080EE0DC080E00BC086EE55
:1021A00009C084EE07C089E205C085E303C08AE266
:1021B00001C081E390E008959091AC0292FF0DC0C0
:1021C000282F2871283019F4877F846006C0282FB3
:1021D0002471243011F48B7F886093FF0DC0282F69
:1021E0002871283119F4877E846106C0282F247154
:1021F000243111F48B7E88612091AD0220FF0DC047
:10220000382F3871383019F4877F816006C0382F35
:102210003171313011F48E7F886021FF0DC0282F7D
:102220002871283119F4877E816106C0282F217119
:10223000213111F48E7E886194FD877E089580E0BF
:1022400008950C947B0D0E9431128FE39CE9019755
:10225000F1F700C000000E94311280E00E945D1181
:1022600080FF04C00E9421110C94901B08950C94CF
:1022700023110E94810D811102C00E94290E0E942B
:102280008C0D80936A020E94940D9093AD0280930E
:10229000AC020E9437110E94900D682F70E080E020
:1022A00090E00E949D076091D2017091D3018091CE
:1022B000D4019091D5010C94D507E82FF0E0EE0FF2
:1022C000FF1FE654FD4F808191810895089580EAB3
:1022D0008A95F1F7089500C008950C946711089548
:1022E0000C946F110C9470110C946F11F894E82FEA
:1022F000E295EF70F0E031A1282F2F7081E090E09F
:1023000001C0880F2A95EAF7982F9095932391A3FF
:1023100092A1892B82A3789408950F931F93CF9352
:10232000DF93CBE8D1E089918F3F11F00E947611C5
:1023300081E0C139D807B9F7CBE7D1E00BE811E06C
:1023400089918F3F11F00E9476110C171D07C1F77C
:10235000DF91CF911F910F910895BF92CF92DF929D
:10236000EF92FF920F931F93CF93DF938C01C62FB1
:10237000D0E0CE0185579E4F6C01FC0190819F3FBC
:1023800009F450C0B62EF894E92FE295EF70F0E012
:1023900081A19F7021E030E001C0220F9A95EAF7F9
:1023A000822B81A382A12095282322A378940E94C6
:1023B0006B11EBE7F1E04BE851E021E030E0E12C7C
:1023C000F12C61916F3F89F0A62FA295AF70B0E01C
:1023D00090968C9190E06F7002C0959587956A9564
:1023E000E2F780FD02C0C90102C080E090E0E82A67
:1023F000F92A220F331F4E175F0719F7F601808164
:102400008F3F11F00E94761161E0E114F10409F4AC
:1024100060E08B2D0E946D11CC0FDD1FC00FD11F0E
:10242000F982E882DF91CF911F910F91FF90EF9099
:10243000DF90CF90BF9008950E948D118CE0EAEB61
:10244000F2E0DF01982F1D929A95E9F7EEEAF2E0AB
:10245000DF011D928A95E9F786E00E947C120C94B8
:102460008502FF920F931F93CF93DF93CDB7DEB713
:102470002C970FB6F894DEBF0FBECDBF8E010F5F55
:102480001F4F8CE0F80111928A95E9F7F12C6F2D1E
:10249000C8010E94AD11F394F6E0FF12F8CF4CE0B2
:1024A00050E0B8018EEA92E00E940F23FF24F394DB
:1024B000009709F4F12C892B41F08CE0F801AEEA89
:1024C000B2E001900D928A95E1F72F2D46E06AEB7C
:1024D00072E08EEA92E00E947D120E9487028F2DA8
:1024E0002C960FB6F894DEBF0FBECDBFDF91CF9113
:1024F0001F910F91FF9008950895FF920F931F93DE
:10250000CF93DF93F82E092F162FD72FC42F222316
:1025100049F081E080936D020E94431B90936C020E
:1025200080936B0280916D028823D9F080916B02B9
:1025300090916C020E945B1B059798F0EF2DF02F95
:10254000A12FBD2F80E090E04C2F50E0841795071D
:1025500034F4219131912D933D930196F7CF109250
:102560006D02DF91CF911F910F91FF9008950E940E
:102570005B1D0E946F0E0C94671D0E946B1D0E94D4
:10258000140F0C94851D0E94E11A0E94421D0E94A6
:102590005B0E0E94B7120E94BD120E94650EFBCF17
:1025A0008091740280FF06C06091090170E0660F9F
:1025B000771F26C081FF04C06091090184E005C037
:1025C00082FF07C06091090188E0689FB001112473
:1025D00017C0909173029923D1F06091080196176A
:1025E00088F72091090188E0289F90011124929F8B
:1025F000A001939F500D112470E0CA010E94B922DE
:102600006038710540F46115710519F406C068E081
:1026100070E0862F08958FE7089581E008958091F6
:10262000740280FF08C06091050170E075956795A0
:102630007595679521C081FF06C06091050170E026
:102640007595679519C082FF04C06091050170E01F
:1026500010C090917202992399F06091040196172D
:10266000A0F780910501899FC001112470E00E94AC
:10267000B9226038710540F46115710519F406C07E
:1026800061E070E0862F08958FE7089581E0089556
:102690008D3E21F40E94D012819504C08E3E29F413
:1026A0000E94D0128093780208958F3E21F40E94F8
:1026B000D012819504C0803F29F40E94D0128093EB
:1026C00077020895893F19F40E940F1305C08A3FCD
:1026D00031F40E940F1381958093790208958B3F06
:1026E00021F40E940F13819504C08C3F29F40E94AD
:1026F0000F1380937A0208959FE0980F983078F432
:1027000021E030E0A90102C0440F551F9A95E2F77D
:10271000CA0190917602892B8093760208958D3FAD
:1027200021F48091740281600BC08E3F21F480916E
:102730007402826005C08F3F29F480917402846026
:102740008093740208958D3E39F49091780297FF3A
:1027500035C01092780259C08E3E29F490917802CB
:102760001916BCF32BC0909177028F3E29F497FF86
:1027700025C01092770249C0803F19F41916CCF396
:102780001DC090917902893F29F41916BCF410926A
:1027900079023BC08A3F19F497FF10C0F8CF8B3FF6
:1027A00039F490917A0297FF09C010927A022DC0F5
:1027B0008C3F21F490917A021916BCF39FE0980F98
:1027C000983080F421E030E0A90102C0440F551F89
:1027D0009A95E2F7CA0180959091760289238093B9
:1027E000760213C08D3F21F4809174028E7F0BC05E
:1027F0008E3F21F4809174028D7F05C08F3F29F4B4
:10280000809174028B7F8093740280917702811192
:1028100006C080917802811102C0109273028091EB
:102820007902811106C080917A02811102C0109252
:10283000720208950E94431B20917702211104C067
:1028400020917802222321F09093710280937002EC
:1028500020917902211104C020917A02222321F0D3
:1028600090936F0280936E0285E792E00C94AF190B
:10287000EF92FF920F931F93CF93DF9300D000D07E
:1028800000D0CDB7DEB786E0E5E7F2E0DE011196D5
:1028900001900D928A95E1F7E0907702F09078022E
:1028A0000091790210917A021092770210927802C8
:1028B0001092790210927A02E11003C0FF2009F40D
:1028C0005DC080917002909171020E945B1BAC010F
:1028D00090917302992339F020910A0130E0241776
:1028E000350758F04BC020910B018AE0289F9001DA
:1028F00011242417350718F041C09F3F19F09F5F3E
:1029000090937302EE2061F00E94D0121E1414F016
:102910009FEF01C091E0989F902D11249093770232
:10292000FF2061F00E94D0121F1414F09FEF01C02D
:1029300091E0989F902D1124909378023091770226
:102940003323E1F0209178022223C1F045EB3403D8
:10295000C0011124992319F09093770203C081E0FC
:102960008093770235EB2303C0011124992319F0DA
:102970009093780203C081E080937802011103C034
:10298000112309F45DC080916E0290916F020E9444
:102990005B1BAC0190917202992339F020910601E2
:1029A00030E02417350758F04BC0209107018AE02A
:1029B000289F900111242417350718F041C09F3F2C
:1029C00019F09F5F90937202002361F00E940F1331
:1029D000101614F09FEF01C091E0989F902D1124E4
:1029E00090937902112361F00E940F13111614F0D5
:1029F0009FEF01C091E0989F902D112490937A024F
:102A0000309179023323E1F020917A022223C1F040
:102A100045EB3403C0011124992319F090937902F6
:102A200003C081E08093790235EB2303C0011124B8
:102A3000992319F090937A0203C081E080937A027F
:102A40008091770281110BC080917802811107C0BB
:102A500080917902811103C080917A0281110E94D4
:102A60001A14EB82FC820D831E8386E0FE013196F0
:102A7000A5E7B2E001900D928A95E1F726960FB690
:102A8000F894DEBF0FBECDBFDF91CF911F910F91A4
:102A9000FF90EF900895E5E7F2E086E0DF011D92F8
:102AA0008A95E9F7109273021092720210927402E2
:102AB000089586E090E00C941C23682F86E090E057
:102AC0000C942A238091C602847089618093C60287
:102AD0000C945D150E94810D811104C00E94290E85
:102AE0000E9462150E9459158093C602282F2695D0
:102AF0002695269530E02430310524F087708861D2
:102B00008093C6028091C60280FF04C08695869598
:102B1000869501C080E00C947B162091C602822F1E
:102B2000869586958695482F50E04330510554F49C
:102B30008F5F982F990F990F990F822F8770892B8C
:102B40008093C6028091C60281608093C6020E9473
:102B50005D158091C6028695869586950C947B16A8
:102B60008091C602982F969596959695A1F0915EC4
:102B7000990F990F990F8770892B8093C602887FD0
:102B800091E009F490E08091C60290FB80F9809377
:102B9000C6020E945D158091C6028695869586952F
:102BA0000C947B168091C60280FD13C081608093D7
:102BB000C602813019F489E08093C6028091C60272
:102BC0000E945D158091C6028695869586950C9427
:102BD0007B1608958091C60280FF08C08E7F809387
:102BE000C6020E945D1580E00C947B1608958091CA
:102BF000C60280FD0C94EA150C94D2159091C60281
:102C0000892F8695869586958F5F8F719770843012
:102C100038F4880F880F880F892B8093C60202C072
:102C20009093C6028091C602887F91E009F490E0FB
:102C30008091C60290FB80F98093C6020E945D15C8
:102C40008091C6028695869586950C947B16843075
:102C500008F083E09091C6029770282F220F220F70
:102C6000220F922B9093C602987F21E009F420E076
:102C70009091C60220FB90F99093C6020C947B16AB
:102C80000E9427168091C6020C945D159C01FB01E1
:102C90008281882349F12E3BFCE53F07C9F040F4CF
:102CA0002C3BECE53E0769F02D3B3C4561F0089577
:102CB000203C9CE5390791F070F0213C3C4589F0BF
:102CC000089583E001C080E00E94401680E00895EE
:102CD0000E94B015FBCF0E948D15F8CF0E94F7150A
:102CE000F5CF0E94FE15F2CF81E00895279A2F9824
:102CF00008952F9808958F929F92AF92BF92CF928E
:102D0000DF92EF92FF920F931F93CF93DF93C82F21
:102D1000843050F4811109C080918000877F8093B6
:102D200080000E94791606C0C3E080918000886010
:102D300080938000A0918600B09187002C2F30E016
:102D40000E94F52223E030E040E050E00E94CD22D6
:102D50000027122F232F342F012F122F232F332739
:102D600080918600909187006CE070E00E94A5221F
:102D70006017710730F0C80169E070E00E94A52279
:102D80005EC08091860090918700E0908600F09070
:102D90008700E0918600F0918700C6E0D0E0BE0198
:102DA0000E94A522060F171F211D311D4801590140
:102DB00085E0880C991CAA1CBB1C8A95D1F7C70119
:102DC000BE010E94A5226F01E12CF12CA701960102
:102DD000260F371F411D511DC501B4010E94CD2290
:102DE00069017A01E0918600F0918700CA01B9017A
:102DF0000E9495229B01AC01DF010E9404239B01EC
:102E0000AC01C701B6010E949522DC01CB012FE085
:102E1000B695A795979587952A95D1F70091860045
:102E20001091870020E030E0081719072A073B07B8
:102E300028F46091860070918700CB01BC017093EB
:102E40008D0060938C00DF91CF911F910F91FF90C7
:102E5000EF90DF90CF90BF90AF909F908F900895AC
:102E600008950E9476168AE08093800089E180931D
:102E700081008FEF9FEF90938700809386000C94E2
:102E80006A15CF93DF93EC01FB018281882309F45B
:102E90003CC1C430FDE5DF0760F4CB3F9CE5D907BA
:102EA00088F49E0122503C452431310508F02EC1A2
:102EB00009C0C236EDE5DE0729F0C63AFDE5DF07B9
:102EC00009F024C10E94940D9093AD028093AC024E
:102ED000C1318CE5D80709F4C6C008F042C0C9303A
:102EE000ECE5DE0709F49BC000F5C5308CE5D8079A
:102EF00009F485C078F4C330ECE5DE0709F478C046
:102F000008F07AC0C230DC4509F0F5C08091AC020F
:102F10008160EFC0C7309CE5D90709F478C008F09C
:102F20007AC08091AC028061E4C0CD30FCE5DF075F
:102F300009F487C058F4CB309CE5D90709F479C06F
:102F400008F07BC08091AC0288606FC0CF30FCE598
:102F5000DF0709F480C008F082C08091AC02877F4F
:102F6000C8C0CE3F9CE5D90709F471C000F5C53152
:102F7000FCE5DF0709F485C068F4C3319CE5D90797
:102F800009F475C008F095C00E9445078091AC0215
:102F90008F77AFC0CC3FFCE5DF07A9F108F054C044
:102FA000CB3FDC4509F0A7C08091AD0240C0C230E4
:102FB000EDE5DE0709F489C058F4C1158DE5D807A1
:102FC00009F45AC008F069C08091AD0282602FC038
:102FD000C236EDE5DE0709F47CC0C63AFDE5DF0741
:102FE00009F481C0C330DD4509F085C080E06EC0C2
:102FF0008091AC0282607DC08091AC0216C080914D
:10300000AC02886076C08091AD0282604FC0809132
:10301000AC0280626EC08091AC0280646AC00E9483
:1030200045078091AC02806864C0846062C08160A2
:103030003DC08091AC028E7F5CC08091AC028D7FE0
:1030400058C08091AC0216C08091AD0218C080912A
:10305000AD028D7F2BC08091AC028F7E4AC08091E3
:10306000AC028F7D46C08091AC028F7B42C08091C4
:10307000AC02877F8B7F3DC08091AD028D7F8E7FBC
:1030800015C08091AC0282FB222720F991E09227A3
:1030900090FB82F990FB83F92CC08091AD02982FB0
:1030A000909591708E7F892B90FB81F98093AD0272
:1030B00022C00E9445078091AC0287FB222720F99D
:1030C00091E0922790FB87F914C081E00E942B0EBB
:1030D00012C08091AC0284FB222720F991E0922754
:1030E00090FB84F906C08091AC02982F909590FBDC
:1030F00080F98093AC028091AC029091AD020E9465
:10310000A50D0E94450780E001C081E0DF91CF91CD
:103110000895CF93DF9386319C4541F5EB010E94E2
:10312000980C982F8A812091020130910301882305
:1031300079F09A7A81E009F480E080937B02911122
:1031400002C069E201C065E3C9010E947F1A0AC09A
:1031500080917B02811102C069E201C065E3C9016F
:103160000E948A1A0E94DA0C80E001C081E0DF919F
:10317000CF9108950F931F93CF93DF93C42FD22F36
:10318000FC0182818823C9F040937E020E94431B88
:1031900090937D0280937C0280E28C0F883008F04F
:1031A00057C0C77081E001C0880FCA95EAF7DF9168
:1031B000CF911F910F910C94A20480917E0248132D
:1031C00030C080917C0290917D020E945B1B883C04
:1031D000910538F510E21D0FCD17B9F080E28C0F84
:1031E000883040F4C77081E001C0880FCA95EAF7C3
:1031F0000E94A904183028F581E09D2F977001C026
:10320000880F9A95EAF70E94A204802F0E949904E1
:103210001830F0F4D77081E001C0880FDA95EAF732
:103220000AC080E28C0F883098F4C77081E001C03A
:10323000880FCA95EAF7DF91CF911F910F910C94F7
:10324000A904802FDF91CF911F910F910C949904C5
:10325000DF91CF911F910F9108950F939C01CB01A6
:10326000243F4CE5340731F188F4293DFCE53F0764
:10327000D9F02A3D4CE5340779F1283D3C45A9F5C4
:1032800006E221EE41EE68ED7CE52BC0263FFCE531
:103290003F07E1F0A8F0273F3C4539F507E225EE6E
:1032A00046EE67EF7CE51DC007E225EE45EE69EDD1
:1032B0007CE517C006E221EE40EE64EF7CE511C02C
:1032C00007E225EE44EE65EF7CE50BC006E221EE59
:1032D00042EE66EF7CE505C008E221E045EE6AEDCE
:1032E0007CE50E94BA1880E008C0FC018281882336
:1032F00019F010927E0201C081E00F910895909321
:1033000093018093920108959093840280938302A5
:103310000895E0918302F0918402309721F00190AA
:10332000F081E02D099480E00895E0918302F0910E
:103330008402309799F020911801222359F02091AE
:10334000AC0227FF07C0DC012C9111962C9311973A
:1033500026E02C930280F381E02D09940895E091FA
:103360008302F0918402309739F022E0DC012C9343
:103370000480F581E02D0994089520918102309117
:1033800082022817390771F090938202809381029C
:10339000E0918302F0918402309721F00680F7815A
:1033A000E02D0994089520917F0230918002281722
:1033B000390771F09093800280937F02E09183023D
:1033C000F0918402309721F00084F185E02D09947A
:1033D0000895FC01329680911801882331F0809184
:1033E000AC0287FF02C09EE101C096E080E09150F0
:1033F00028F021912223D9F38F5FF9CF0895662316
:1034000051F1209118012223E9F02091AC0227FF0D
:1034100019C0462F4695469546954E31E0F46770A3
:1034200021E030E002C0220F331F6A95E2F7FC0171
:10343000E40FF11D828190E02823392381E0232BC2
:1034400069F409C0FC01329608962191621729F0AF
:10345000E817F907D1F780E0089581E008959C010D
:10346000FC0132969FEF80E04191461789F09F3F23
:1034700019F4411101C0982F8F5F8630A9F79F3F43
:1034800039F0F901E90FF11D97FDFA95628308956E
:1034900008959C012A5F3F4FFC014281461301C001
:1034A0001282019682179307B9F70895262F269561
:1034B000269526952E3168F4FC01E20FF11D677008
:1034C00021E030E001C0220F6A95EAF78281282BC3
:1034D00022830895262F2695269526952E3170F461
:1034E000FC01E20FF11D677021E030E001C0220F06
:1034F0006A95EAF7209582812823228308952091F6
:103500001801222329F02091AC0227FD0C94561AB1
:103510000C942F1A20911801222329F02091AC023B
:1035200027FD0C946A1A0C94491A20911801FC0189
:103530003296222331F08091AC0287FF02C08EE1E7
:1035400001C086E0DF011D928A95E9F7089508958C
:103550000C94A71A83E0809385020C94A81A811119
:1035600002C081E001C082E0809385020C94A81A19
:103570000C94AF1A81E0809385020C94A81A0C94E5
:10358000BA1A08950C94C11A0C94C21A0C94C11A58
:103590000C94C11A0C94C11ACF930E94C81A0E94AD
:1035A00031120E94C61AC0E08C2F0E945D11892B37
:1035B00029F4CF5FC630C1F780E001C081E0CF9130
:1035C000089508951F920F920FB60F9211248F93B2
:1035D0009F93AF93BF9380918602811113C0809116
:1035E000C7029091C802A091C902B091CA02419647
:1035F000A11DB11D8093C7029093C802A093C90278
:10360000B093CA02BF91AF919F918F910F900FBE5F
:103610000F901F9018958091CF02843031F10E9455
:10362000F2021092860220E488E190E00FB6F8944E
:10363000A895809360000FBE2093600083B7817FC0
:10364000846083BF83B7816083BF7894889583B794
:103650008E7F83BF0FB6F894A89580916000886133
:1036600080936000109260000FBE08950E9445078D
:103670000C94F90282E084BD93E095BD9AEF97BD6A
:1036800080936E0008952FB7F8948091C7029091AF
:10369000C802A091C902B091CA022FBF08952FB7E6
:1036A000F8946091C7027091C8028091C90290910C
:1036B000CA022FBF08959C014FB7F8948091C702AA
:1036C0009091C802A091C902B091CA024FBF821B5B
:1036D000930B089578941F920F920FB60F921124B6
:1036E0008F939F93AF93BF938091C7029091C8022D
:1036F000A091C902B091CA020196A11DB11D80938B
:10370000C7029093C802A093C902B093CA02BF91A6
:10371000AF919F918F910F900FBE0F901F901895B2
:1037200081E08093E00080E28093D8001092C9008D
:103730008FE19EE40197F1F700C0000087E090EB75
:10374000DC018093D8029093D902A093DA02B0935F
:10375000DB029CE088E10FB6F894A89580936000A6
:103760000FBE90936000FFCF8091AA020895089544
:1037700022E02093E9002FEF3091E800215035FD41
:1037800006C035ED3A95F1F700002111F5CF2091F3
:10379000E80025FF0BC040E050E066E070E00E94CA
:1037A000F71D8091E8008E778093E8000895CF930D
:1037B000DF9320911801222339F02091AC0227FFDA
:1037C00003C060E222E002C068E021E02093E9004B
:1037D0002FEF3091E800215035FD06C035ED3A95C8
:1037E000F1F700002111F5CF2091E80025FF1DC061
:1037F000EC0180911801811105C040E050E068E0C3
:1038000070E003C070E040E050E0CE010E94F71D80
:103810008091E8008E778093E80080E2FE01AAE8BC
:10382000B2E001900D928A95E1F7DF91CF91089572
:103830008093870270938902609388028091CF02FF
:10384000843001F582E08093E9008FEF9091E800E9
:10385000815095FD06C095ED9A95F1F70000811114
:10386000F5CF8091E80085FF0DC040E050E063E0B7
:1038700070E087E892E00E94F71D8091E8008E7763
:103880008093E8000895BC0184E00C94181CBC01EE
:1038900083E00C94181C8091CE02811109C00E9413
:1038A000881F0E94E51F8091E20084608093E200FF
:1038B00008951092CE0208950C94BF1A6091CB0225
:1038C00081E0611101C080E00C94AA1A9091CF02AE
:1038D00081E0943009F080E06091CB020C94AF1A43
:1038E00042E061EC81E00E94011F42E261EC82E073
:1038F0000E94011F9091CF0281E0943009F080E096
:103900006091CB020C94B81A8091D102833009F4F3
:1039100061C030F4813071F0823009F49AC00895AA
:103920008A3009F486C08B3009F46CC0893009F004
:10393000A8C020C08091D002813A09F0A2C0809135
:10394000E800877F8093E8008091D4029091D502AF
:10395000892B21F460E28AE892E003C060E080E015
:1039600090E070E00E94421E8091E8008B77809387
:10397000E80008958091D002813209F082C08091E0
:10398000D4029091D502029708F07BC08091E800A4
:10399000877F8093E8008091E80082FD05C08091D8
:1039A000CF028111F8CF6DC02091F3008091F20019
:1039B00090E0922B029731F48091F100813011F068
:1039C000863021F48091F1008093AA028091E80072
:1039D0008B7753C08091D002813A09F052C0809118
:1039E000D4029091D502892B09F04BC08091E80058
:1039F000877F8093E8008091E80080FFFCCF809172
:103A0000180136C08091D0028132D9F58091D4025C
:103A10009091D502892BA9F58091E800877F80934A
:103A2000E8000E94361F8091D202809318010C9406
:103A300045078091D002813221F58091E800877F8F
:103A40008093E8000E94361F8091D3028093AB02DE
:103A500008958091D002813AA1F48091E800877F97
:103A60008093E8008091E80080FFFCCF8091AB025A
:103A70008093F1008091E8008E778093E8000C94A9
:103A8000361F089584B7877F84BF0FB6F894A89532
:103A900080916000886180936000109260000FBE8A
:103AA00090E080E80FB6F8948093610090936100F5
:103AB0000FBE0C94BA1A0E94881F0E94E51FE2EE06
:103AC000F0E080818460808378940C947A228CE08A
:103AD00091E00C9484198091CF028530A9F48091F3
:103AE000CF02853079F40E940B1B8091CD02882390
:103AF000B1F30E94CC1A882391F30E94E11D0E9429
:103B00004507EDCF0C94361B089508950C94881D3D
:103B1000292F332723303105C9F060F421303105D6
:103B200081F02230310509F044C08BE390E02EE8AB
:103B300032E043C021323105E1F02232310549F152
:103B400038C082E190E029EC32E037C0992781301B
:103B5000910549F028F0029761F5E8E5F2E005C02B
:103B6000EAE8F2E002C0E8E7F2E0849190E09F0129
:103B700024C06115710541F061307105D1F489E00F
:103B800090E029EB32E019C089E090E020EA32E0D1
:103B900014C06115710541F06130710551F486EB77
:103BA00090E02BED32E009C080E490E021E933E0C1
:103BB00004C080E090E020E030E0FA01318320830F
:103BC000089580E189BD82E189BD09B400FEFDCF81
:103BD0008091D8008F7D8093D8008091E000826032
:103BE0008093E0008091E00081FDFCCF0895CF92AA
:103BF000DF92EF92FF920F931F93CF93DF93EC012D
:103C00008B017A010E94551F811133C0E114F10428
:103C100039F0F70180819181081B190BC80FD91F5A
:103C2000C12CD12C0115110519F18091E80085FDF9
:103C300016C08091E8008E778093E800E114F104CB
:103C400049F0F70180819181C80ED91ED182C082CE
:103C500085E00FC00E94551F882321F30AC0899177
:103C60008093F10001501109FFEFCF1ADF0ADACF7C
:103C700080E0DF91CF911F910F91FF90EF90DF9047
:103C8000CF9008952091D6023091D702261737079A
:103C900048F06115710539F42091E8002E772093E2
:103CA000E80001C0B901FC0120E06115710579F15E
:103CB0008091CF028823F1F18530F1F18091E80005
:103CC00083FD3CC08091E80082FD2EC08091E80019
:103CD00080FFEBCF2091F3008091F20090E0922BD7
:103CE0006115710551F08830910538F421912093C8
:103CF000F100615071090196F3CF21E0089709F0B6
:103D000020E08091E8008E778093E800CECF2111EB
:103D1000CFCF0AC08091CF02882361F0853061F057
:103D20008091E80083FD0AC08091E80082FFF2CF15
:103D300080E0089582E0089583E0089581E0089589
:103D40002091D6023091D7022617370748F0611527
:103D5000710539F42091E8002E772093E80001C026
:103D6000B901FC0120E06115710591F18091CF024C
:103D7000882309F440C0853009F43FC08091E800F1
:103D800083FD3DC08091E80082FD2FC08091E80056
:103D900080FFE9CF2091F3008091F20090E0922B18
:103DA0006115710559F08830910540F424912093F4
:103DB000F1003196615071090196F2CF21E0089728
:103DC00009F020E08091E8008E778093E800CBCF67
:103DD0002111CCCF0AC08091CF02882361F08530B9
:103DE00061F08091E80083FD0AC08091E80082FFC5
:103DF000F2CF80E0089582E0089583E0089581E0A5
:103E00000895982F973068F59093E900981739F046
:103E10007091EC002091ED005091F00003C0242F30
:103E2000762F50E021FD02C09F5FECCF3091EB0078
:103E30003E7F3093EB003091ED003D7F3093ED00FD
:103E40003091EB0031603093EB007093EC002093E5
:103E5000ED005093F0002091EE0027FDE5CF80E0CB
:103E600008958F708093E90081E008958091D002D9
:103E700087FF11C08091E80082FD05C08091CF02CC
:103E80008111F8CF11C08091E8008B770BC0809131
:103E9000CF02882349F08091E80080FFF8CF80911D
:103EA000E8008E778093E80008952091E400309137
:103EB000E50095E64091EC00842F817040FF23C01F
:103EC0008091E80080FD1DC08091CF02882399F089
:103ED000853099F08091EB0085FD11C04091E400A0
:103EE0005091E5002417350729F3915011F09A01FC
:103EF000E1CF84E0089582E0089583E0089581E0B1
:103F0000089580E008954091E80042FFDDCF0895D4
:103F10000E94F61F0E94FE1FE0EEF0E080818160AB
:103F20008083E8EDF0E080818F77808319BCA7ED76
:103F3000B0E08C918E7F8C9380818F7E80831092F5
:103F4000CE0208950F931F93CF93DF930E94F61F25
:103F50000E94FE1FC8EDD0E088818F77888388811A
:103F60008068888388818F7D888319BC1092CF02F6
:103F70001092CB021092CD021092CC0200EE10E013
:103F8000F80180818B7F808388818160888342E013
:103F900060E080E00E94011FE1EEF0E080818E7F12
:103FA0008083E2EEF0E080818160808380818860A0
:103FB0008083F80180818E7F8083888180618883FF
:103FC000DF91CF911F910F910895E8EDF0E080818E
:103FD0008F7E8083E7EDF0E080818160808384E0E4
:103FE00082BF81E08093CE020C94A21FE8EDF0E046
:103FF00080818E7F80831092E20008951092DA0013
:104000001092E10008951F920F920FB60F921124A3
:104010002F933F934F935F936F937F938F939F93D0
:10402000AF93BF93EF93FF938091E10082FF0BC0AA
:104030008091E20082FF07C08091E1008B7F809336
:10404000E1000E9479228091DA0080FF1FC08091F8
:10405000D80080FF1BC08091DA008E7F8093DA0049
:104060008091D90080FF0DC080E189BD82E189BDCA
:1040700009B400FEFDCF81E08093CF020E944B1C6B
:1040800005C019BC1092CF020E94591C8091E1001A
:1040900080FF19C08091E20080FF15C08091E2008E
:1040A0008E7F8093E2008091E20080618093E20045
:1040B0008091D80080628093D80019BC85E08093FD
:1040C000CF020E945E1C8091E10084FF30C080918D
:1040D000E20084FF2CC080E189BD82E189BD09B482
:1040E00000FEFDCF8091D8008F7D8093D800809115
:1040F000E1008F7E8093E1008091E2008F7E8093CB
:10410000E2008091E20081608093E2008091CB0226
:10411000882311F084E007C08091E30087FD02C08E
:1041200081E001C083E08093CF020E94661C8091F1
:10413000E10083FF29C08091E20083FF25C08091C8
:10414000E100877F8093E10082E08093CF021092AC
:10415000CB028091E1008E7F8093E1008091E200AC
:104160008E7F8093E2008091E20080618093E20084
:1041700042E060E080E00E94011F8091F0008860D2
:104180008093F0000E945C1CFF91EF91BF91AF9172
:104190009F918F917F916F915F914F913F912F915F
:1041A0000F900FBE0F901F9018951F920F920FB691
:1041B0000F9211242F933F934F935F936F937F93AD
:1041C0008F939F93AF93BF93CF93DF93EF93FF931F
:1041D000C091E900CF708091EC00D82FD17080FDA4
:1041E000D0E81092E9008091F000877F8093F00082
:1041F00078940E9419211092E9008091F000886063
:104200008093F000CD2BCF70C093E900FF91EF9128
:10421000DF91CF91BF91AF919F918F917F916F91DE
:104220005F914F913F912F910F900FBE0F901F9074
:1042300018951F93CF93DF93CDB7DEB7AA970FB62C
:10424000F894DEBF0FBECDBFE0EDF2E08091F1004B
:10425000819322E0E83DF207C9F70E94841C809117
:10426000E80083FF2EC18091D0029091D102492FA6
:1042700050E04A30510508F024C1FA01EE59FF4FD1
:104280000C94EF22803821F0823809F01AC108C05E
:104290008091CC029091CD02992389F082600FC069
:1042A0008091D4028F70873008F00BC18093E900B1
:1042B0008091EB0085FB882780F91092E9009091AE
:1042C000E800977F9093E8008093F1001092F1004E
:1042D000D1C0282F2D7F09F0F4C0882319F0823037
:1042E00061F0EFC08091D202813009F0EAC09330D2
:1042F00009F080E08093CD022EC08091D20281111E
:104300002AC08091D4028F702FEF280F263008F03A
:10431000D8C08093E9002091EB0020FF1CC09330AF
:1043200021F48091EB00806214C09091EB009061C9
:104330009093EB0021E030E0A90102C0440F551F2B
:104340008A95E2F74093EA001092EA008091EB0030
:1043500088608093EB001092E9008091E800877FED
:104360008093E8000E94361FACC08111AAC0109152
:10437000D2021F778091E3008078812B8093E30045
:104380008091E800877F8093E8000E94361F80912B
:10439000E80080FFFCCF8091E30080688093E30019
:1043A000111102C082E001C083E08093CF0289C076
:1043B0008058823008F085C08091D2029091D3025B
:1043C0008C3D53E0950779F583E08A838AE28983FF
:1043D0004FB7F894DE01139620E03EE051E2E32F60
:1043E000F0E050935700E49120FF03C0E295EF7096
:1043F0003F5FEF708E2F90E0EA3010F0C79601C05B
:10440000C0968D939D932F5F243149F74FBF8091C4
:10441000E800877F8093E8006AE270E0CE010196B1
:104420000E94421E16C06091D4027091D502AE0166
:104430004F5F5F4F0E94861DBC01892B09F441C06C
:104440009091E800977F9093E80089819A810E947B
:10445000A01E8091E8008B778093E80032C08038FE
:1044600081F58091E800877F8093E8008091CB02FE
:104470008093F1008091E8008E7772CF811121C086
:104480008091D2029091D30299270297D4F480911F
:10449000E800877F8093E8008091D2028093CB026E
:1044A0000E94361F8091CB02811106C08091E300EB
:1044B00087FD02C081E001C084E08093CF020E94AA
:1044C000701C8091E80083FF0AC08091E800877F1C
:1044D0008093E8008091EB0080628093EB00AA96C5
:1044E0000FB6F894DEBF0FBECDBFDF91CF911F9105
:1044F00008950895CF938091CF028823A1F0C091B1
:10450000E900CF709091EC00892F817090FD80E8D8
:10451000C82B1092E9008091E80083FD0E941921C8
:10452000CF70C093E900CF910895DB018F939F93E3
:104530000E940423BF91AF91A29F800D911DA39F64
:10454000900DB29F900D11240895AA1BBB1B51E141
:1045500007C0AA1FBB1FA617B70710F0A61BB70BF3
:10456000881F991F5A95A9F780959095BC01CD0198
:10457000089597FB072E16F4009407D077FD09D015
:104580000E94A52207FC05D03EF4909581959F4F8F
:104590000895709561957F4F0895A1E21A2EAA1B88
:1045A000BB1BFD010DC0AA1FBB1FEE1FFF1FA217E3
:1045B000B307E407F50720F0A21BB30BE40BF50BE0
:1045C000661F771F881F991F1A9469F76095709569
:1045D000809590959B01AC01BD01CF010895EE0F30
:1045E000FF1F0590F491E02D0994A29FB001B39FA5
:1045F000C001A39F700D811D1124911DB29F700DEC
:10460000811D1124911D08950E94F522A59F900DF2
:10461000B49F900DA49F800D911D11240895FB015E
:10462000DC0104C08D910190801921F4415050406B
:10463000C8F7881B990B0895F999FECF92BD81BDEB
:10464000F89A992780B50895A8E1B0E042E050E0DB
:104650000C945023262FF999FECF92BD81BDF89A74
:10466000019700B4021639F01FBA20BD0FB6F894B6
:10467000FA9AF99A0FBE08950396272F0E942B23CA
:104680000E942A23252F0E942B23242F0C942B23B6
:104690000196272F0E942B230C942A23DC01CB01A7
:1046A000FC01F999FECF06C0F2BDE1BDF89A319642
:1046B00000B40D9241505040B8F70895F894FFCFE0
:1046C000C8003402280850011E0A1401B41BD71B6D
:1046D000B81B471C431CB71B01E200E900EA00B508
:1046E00000B600B700CD008301CC008A019201948E
:1046F000012102230224022502260227022A02B3F4
:1047000000B4006F007000818283E200E900EA00DB
:10471000B500B600B700CD008301CC008A0192013C
:1047200094012102230224022502260227022A02E2
:10473000B300B4006F0070008182836667F7F6F5FE
:10474000F4F1F09293959496973435303132339159
:02475000360031
:00000001FF
